:1000000010C01FC01EC01DC01CC01BC01AC019C01C
:1000100018C017C016C015C014C013C012C011C03C
:1000200010C011241FBECFE5D1E0DEBFCDBF20E060
:10003000A0E6B0E001C01D92A436B207E1F701D1FD
:100040002CC1DECFDC01FA0110828C918623E9F706
:100050008CE18A95F1F7000088E38A95F1F700C0FA
:100060008C91862319F080818160808388E38A9552
:10007000F1F700C08C91862319F080818260808323
:1000800088E38A95F1F700C08C91862319F080816E
:100090008460808388E38A95F1F700C08C91862381
:1000A00019F080818860808388E38A95F1F700C029
:1000B0008C91862319F080818061808388E38A9502
:1000C000F1F700C08C91862319F0808180628083D3
:1000D00088E38A95F1F700C08C91862319F080811E
:1000E0008064808388E38A95F1F700C08C91862331
:1000F00019F080818068808388E38A95F1F700C0D9
:100100008CE18A95F1F700000895FC019081862F1B
:1001100080959823908398E39A95F1F700C0908199
:1001200040FF02C0962B01C09823908398E39A95D4
:10013000F1F700C0908141FF02C0962B01C09823C7
:10014000908398E39A95F1F700C0908142FF02C036
:10015000962B01C09823908398E39A95F1F700C0FD
:10016000908143FF02C0962B01C09823908398E3AF
:100170009A95F1F700C0908144FF02C0962B01C010
:100180009823908398E39A95F1F700C0908145FFFA
:1001900002C0962B01C09823908398E39A95F1F7BB
:1001A00000C0908146FF02C0962B01C09823908327
:1001B00098E39A95F1F700C047FF04C08081862B31
:1001C000808303C090819823908388E38A95F1F718
:1001D00000C08081862B808398E39A95F1F700C058
:1001E00088E38A95F1F700C00895FF920F931F935B
:1001F000CF93DF938C01F62EEA01109263001092E8
:100200006200E0916200F0916300EC0FFD1F4081FD
:100210006F2DC8017ADF20916200309163002F5F5B
:100220003F4F3093630020936200FE01E20FF31F03
:1002300080818111E6CFDF91CF911F910F91FF90C7
:10024000089580E886BD16BCD99AD19AD29AD398DF
:10025000DA98109261001092600080916000909195
:10026000610001969093610080936000CB9BF5CF75
:100270002FE78AE196E0215080409040E1F700C0EE
:100280000000DA9A2FE78AE196E021508040904002
:0E029000E1F700C00000DA98E0CFF894FFCF4D
:00000001FF
